:10000000ABC0C5C0F7CCC3C0C2C0C1C0C0C0BFC0B8
:10001000A4CCBDC0BCC0BBC0DECCB9C0B8C03230FF
:1000200032323037323530363132000000000000D5
:1000300000000000000000000000000000000000C0
:1000400000000000000000000000000000000000B0
:1000500000000000000000000000000000000000A0
:100060000000000000000000000000000001030488
:10007000050708090B0C0E0F1113141618191B1D78
:100080001F21232527292B2D30323437393B3E4081
:100090004346484B4E5154575A5D606366696D70D4
:1000A00073777A7E8185898D9094989CA0A5A9AD5F
:1000B000B1B6BABFC3C8CDD1D6DBE0E5EAEFF4FAFA
:1000C000FF010102020303040405060708090A0CE4
:1000D0000D0E0F11131416181A1D1F2224272A2D76
:1000E0003033373B3E42464B4F54595D63686E7325
:1000F000797F868C939AA1A8B0B8C0C8D1D9E2EC18
:10010000F5FFFFFFFFFFFFFFFFFFFFFFFFFFFFFF09
:10011000FFFFFFFFFFFFFFFFFFFFFFFFFFFFFFFFEF
:10012000FFFFFFFFFFFFFFFFFFFFFFFFFFFFFFFFDF
:10013000FFFFFFFFFFFFFFFFFFFFFFFFFFFFFFFFCF
:10014000FFFFFFFFFFFFFFFFFFFFFFFFFFFFFFFFBF
:10015000FFFFFFFFFFFF000011241FBECFE5D2E02D
:10016000DEBFCDBF10E0A0E6B0E0E0ECFFE102C0F2
:1001700005900D92A639B107D9F721E0A6E9B0E0C4
:1001800001C01D92A034B207E1F743DC17CF38CF8E
:10019000482F9B01EDE0F1E080E090E05081552395
:1001A00031F00196339680319105C1F709C063E0C3
:1001B00070E0A6DEFC01E35FFE4F408332832183C3
:1001C00008950F931F93CF93DF93D0910D01DD23FB
:1001D00051F100910E0110910F01C091EA00C15040
:1001E000C7FD0DC0EC2FEE0FFF0BE551FF4F019047
:1001F000F081E02DB8018D2F09958111F0CFEDE050
:10020000F1E0838180838481958192838183339619
:1002100081E0EA33F807A9F710923A0110923C0105
:1002200010923B01D2CFDF91CF911F910F91089592
:10023000BC0180913F01ACCF10923F0110923E0172
:1002400010923D0181E08093C400089590E822E07F
:1002500048EA57E030E0815070F00FB6F89496BD50
:1002600026BD0FBEFA013197F1F70FB6F89496BD8F
:1002700036BD0FBEF0CF089586B383FB882780F983
:1002800091E089278093E3000895E0916600F09162
:1002900067003196FB70F460F0936700E0936600AE
:1002A0008091DF008B5A8093DF00E4918091DF0022
:1002B0008E0F0895CF93DF9300D000D000D0CDB73C
:1002C000DEB79091BD002091FB003091FC002751DA
:1002D000364009F492E0843019F46093BE0021C0E6
:1002E0006623F9F0823019F427E9261B622F26E0F5
:1002F000EFE7F0E0DE01119601900D922A95E1F70B
:10030000E82FF0E03197EE0FFF1F21E030E02C0FD7
:100310003D1FE20FF31F0190F081E02DE90FF11D69
:10032000608326960FB6F894DEBF0FBECDBFDF9177
:10033000CF910895BF92CF92DF92EF92FF920F93E9
:100340001F93CF93DF93EC014091BD00E0917A00C1
:10035000EE2311F082E001C0842F90E0DC01AC5864
:10036000BF4F2C9120937800DC01AF58BF4F8C9188
:1003700080937700F0E0E259FF4F3181622F70E007
:10038000442349F0313039F49B01280F311DC90154
:100390009595879536C0C617D70794F1682F70E0FA
:1003A0006C177D0774F1411102C08C2F2AC0821B8B
:1003B000032F10E001501109E82EF12CC701B801FC
:1003C000D0DD6093BB006695E62FF0E0822FC12C54
:1003D000D12CB12CB316A9F0C601B801AEDD822F25
:1003E000860FCE0CDF1CAE01481B510957FF03C01E
:1003F000519541955109E417F5071CF4B394EACFE0
:10040000822FDF91CF911F910F91FF90EF90DF909E
:10041000CF90BF90089581E00895611160937D00B1
:100420000895662389F0813061F48091FE009091F7
:10043000FD00891B681B6093FD0082E080937E00B5
:1004400003C0635E60937C0080917C00873418F069
:1004500086E480937C0008956093B60008950F931E
:100460001F93CF93DF938091BD008093C60080914E
:1004700074008093C700809171008093C8008091C0
:1004800075008093C900809172008093CA008091AA
:100490006F008093CB00809176008093CC00809198
:1004A00073008093CD00809170008093CE00809186
:1004B0007A008093CF008091BE008093D00080911D
:1004C000BC008093D100809179008093D20080910C
:1004D000C0008093D3008091BF008093D4008091AE
:1004E0006B008093D500809169008093D600809145
:1004F0006A008093D700809168008093D800809133
:100500006C008093D90080917C008093DA00809108
:10051000FD008093DB0080917D008093DC00809162
:100520006D008093DD008091B6008093DE00F8942A
:1005300006EC10E0C1E0D1E0F80161918F01CE013D
:100540002BDD2196CA31F1E0DF07B1F765EA80E0E3
:1005500091E022DD7894DF91CF911F910F91089562
:10056000CF93DF9380917B008093C500F894C09176
:10057000C200D091C3006FEFCE010EDD6FEFCE0150
:1005800001960ADD2296CF3FD10510F0C0E0D0E001
:10059000D093C300C093C20065EACE01FDDC609138
:1005A000C500CE010196F8DC7894DF91CF910895D3
:1005B000882321F0813029F4BC9804C0BC98C498E9
:1005C0000895BC9AC49A0895CF93C82F8093E100F0
:1005D0008093E0008091E20081110AC091E0C11196
:1005E00001C090E081E0C23408F480E0890FE0DFD0
:1005F000C11103C019BC18BC0DC0C1508C2F90E0B4
:10060000FC01EF53FF4FE491E9BDFC01E55DFF4FB5
:10061000E491E8BD8091E100853010F492E005C0DE
:100620008E3010F491E001C090E080E80FB6F894AD
:1006300086BD96BD0FBECF9108958093C100C4CFF3
:10064000CF93C091E10089E18C0F873908F080E0F9
:10065000BBDF82E0FBDD8C2FCF91B6CFCF93C09173
:10066000E10080E0B1DF83E0F1DD8C2FCF91ACCFF2
:10067000813019F41092C0000895823019F460930B
:10068000BF000895833019F46093BC00089584304E
:1006900011F4609379000895909100019D3110F458
:1006A00080E009C08370833039F46F70E62FF0E08A
:1006B000EB57FF4F80817CCF0895CF93C0917A0094
:1006C000C11149C0883039F41092BA001092B800B4
:1006D0001092B70041C0813B59F48091BA0081501B
:1006E0008330C8F583E08093BA008093B90033C0AB
:1006F000853BA9F4CB016EE370E01FDC892B61F52B
:100700008091BA008A3F40F58B5F8093BA00809356
:10071000B9001092B8001092B70092DF1DC081306E
:10072000D1F48091B7009091B800019688382EE0FE
:10073000920728F49093B8008093B7000DC01092F0
:10074000B8001092B7008091BA00882329F0815038
:100750008093BA0001C0C1E08C2FCF910895FF9221
:100760000F931F93CF93DF938C01EB01F42E8091B5
:10077000FB009091FC00892B31F0E091FB00F0919F
:10078000FC0089E009951093FC000093FB00012B0D
:1007900039F0E091FB00F091FC00BE018F2D09952E
:1007A00081E08093C400DF91CF911F910F91FF9062
:1007B0000895CF93DF93E091EA00EE2359F0E150E2
:1007C000E093EA00F0E0EE0FFF1FE551FF4FC0811C
:1007D000D18102C0C0E0D0E0E091EA00EE2341F018
:1007E000F0E0EE0FFF1FE751FF4F8081918102C0C3
:1007F00080E090E04AE060E070E0B1DFCE01DF91A0
:10080000CF910895883029F41092B30010929A0085
:1008100015C08130F9F490919A00911107C06032AF
:10082000710568F180939A0007DD29C0913081F449
:100830006B3B710528F082E080939A0080E01EC037
:1008400061157105E1F06270862F880F8E5E16C00B
:10085000B0DF15C0813811F0813E89F491E09093AA
:100860009A00813E21F48091B300865F03C080919D
:10087000B3008F5F8093B300DFDC8BE4A5DE80E004
:1008800008959C019091EA00983088F4E92FF0E0F7
:10089000EE0FFF1FE551FF4F318320839F5F909341
:1008A000EA0048E0C9015BDF8091EA0008958FEF1C
:1008B00008950F931F93CF93DF93EC018B0179DFA2
:1008C000B801CE01DF91CF911F910F91DACF843023
:1008D00011F58091FB009091FC002AE0823F920785
:1008E00029F469E170E08EEB96E013C08E5B9640D0
:1008F00061F49091E100923040F0892F86959695B1
:100900009695890F9ADE80E0089560E070E08EEEA3
:1009100094E0CFDFF8CF81E00895813C29F460E0D6
:1009200070E08EEE94E006C0823C31F460E070E04E
:1009300084EB94E0BEDF14C0813B41F4CB016EE355
:1009400070E0FBDA892B61F47BDE0AC0813E51F452
:10095000CB016EE370E0F1DA6F5F60936C007FDDD6
:1009600080E0089581E00895CF93C0917A00C1118D
:1009700017C0813C29F460E070E08EEE94E006C080
:10098000823C31F460E070E084ED94E092DF09C0D5
:10099000873B31F460E070E08FE196E072DF01C0E8
:1009A000C1E08C2FCF910895813C29F460E070E084
:1009B0008EEE94E006C0823C31F460E070E08DE899
:1009C00094E077DF07C0873B39F460E070E083E2B2
:1009D00096E057DF80E0089581E00895CF93DF939C
:1009E000EB01883079F480E0EFDD80916D00837059
:1009F000DFDD1092BA00CD2B19F481E08093E20084
:100A0000C0E0C9C0813051F469317105C8F38093E9
:100A1000E20080916D008370CBDDF2CF8330F9F47A
:100A20002091C000222359F08091BF0090E062EC39
:100A300071E066DAC817D90710F020937B006C2F9D
:100A400080916D0029DE8091B6008823C9F290E084
:100A500062EC71E055DA8C179D0790F64BC0813B34
:100A600089F481E090E066DCAFDD8091BC0081110B
:100A7000C7CF8091BD00811102C0689708F261E084
:100A800070E028C0813ED9F3813821F480917B0049
:100A900090E013C0813C21F46091E10070E01AC045
:100AA000823B79F48091790090917A009111809144
:100AB000BE00811104C086E990E03CDC05C086E9F7
:100AC00003C0823E19F480E07FDD9ACF823C31F48E
:100AD00066E970E08EEB96E0ECDE92CF833999F315
:100AE000833C29F460E070E084EB94E0F5CF843C33
:100AF00031F4A6DD60E070E08BE296E0EDCF8D3B57
:100B000031F4F89488ED81BD7894A895FFCF8F3C9F
:100B100029F460E070E08BE092E0DECF8A3B81F464
:100B2000CD2B19F5C0917A00CC2321F089DD1092EC
:100B30007A0019C060E070E087E196E0A2DE2BC089
:100B4000833B29F460E070E082EF9AE0C5CF873CF8
:100B500061F490916D0081E0890F83709C7F982BE8
:100B600090936D0025DD7BDC4BCFC0917A00C111E5
:100B700011C08A3C31F464DD81E080937A006FDC3F
:100B80000AC0853C39F45CDD60E070E089E69CE0F9
:100B900090DE01C0C1E08C2FDF91CF9108958830A5
:100BA00061F410929B0080E00FDD8091E3008111E1
:100BB00036C081E080939B0022C0982F907F903BAD
:100BC000B1F420919B00421778F0CB016DE570E005
:100BD000B4D9029739F42F5F20939B004217F8F0A5
:100BE00088E303C082E101C080E0EEDC18C0903EE3
:100BF00061F480919B00882389F0481778F060E0C9
:100C000070E082E094E03DDE0AC08A3041F46091F9
:100C1000B30080919B00F901099521DCCADD80E0D9
:100C200008954091BD004E5F2AE531E0B8CF2AE536
:100C300031E044E0B4CF28E333E044E0B0CF2DE02E
:100C400032E041E0ACCF21E132E042E0A8CF2CE23B
:100C500032E041E0A4CF0F931F93CF93DF93D82FBF
:100C60008B0180798039B1F42091740090917500E6
:100C70008D2F8F70823041F48091C000811108C0A7
:100C8000822F291728F403C0822F921708F4892F86
:100C90009BDC1BC0803819F480E096DC08C0D8309B
:100CA00031F480916D008695869582DC3FC0D1300D
:100CB00061F40931110508F458C0D093E200809125
:100CC0006D008695869574DC50C0D33039F48091E0
:100CD0006D00602F86958695DFDC47C0D33C31F4EC
:100CE000AFDC60E070E08EEE94E00AC0D43C89F4A2
:100CF000C091C000CC2331F06C2F70E08EEB96E0F9
:100D0000D8DD33C060917B0070E08EEB96E0D1DDE2
:100D10002FC0D43B31F4A2DC10923F0161E070E0BF
:100D2000EDCFD53C19F466E970E0E8CFC0917A00C8
:100D3000C1111DC0DA3B31F460E070E087E296E05B
:100D4000A0DD16C0D73C99F490916D00892F86954F
:100D500086958F5F8370282F220F220F9370920F3A
:100D600090936D0025DC7BDB03C0C0E001C0C1E0D7
:100D70008C2FDF91CF911F910F9108959F92AF9289
:100D8000BF92CF92DF92EF92FF920F931F93CF9378
:100D9000DF93182FEB0190907800B0907700D090FF
:100DA000BD00DD2019F0A090BB0002C0AA24A394CE
:100DB000E090790000917A000111E090BE00EE20F1
:100DC00051F081E0E81621F080917B008B1518F03E
:100DD000A6E9FA2E01C0FB2CC090BA00BE01812FFB
:100DE0006CDC6091BA00662339F0C1100CC08091B0
:100DF000E10080939E0007C0CC2029F060E070E005
:100E00008EEE94E038C0812F8D7F8830D1F410921F
:100E1000B5001A3019F4C0917B00D0E0892D90E024
:100E20008C179D0738F48B2D90E0C817D90710F464
:100E3000C0937B00CE017EDA00DC81E08093650008
:100E400025C1113CD9F2123C71F48091E1008F155B
:100E500010F48F2D02C080917B00EFDB8091E100C8
:100E600080939E0013C1143C41F480E0ADDB60E050
:100E700070E08BE296E01DDD09C18FE4810F8230C6
:100E8000B8F5DD2039F0CE0168E170E056D8892B45
:100E900009F0FCC08091E100209761F4123B11F44D
:100EA0008FEF05C08B15E0F79816A8F081E08093CE
:100EB000650011C0C733E1E0DE0768F08B1580F7ED
:100EC000CD36D24040F0981630F0BADB60E070E0EA
:100ED0008BE296E0EEDC809165006A2D70E0082ED2
:100EE000000C990B0DD82091E100820F911DEDC0EF
:100EF0008FE1810F823038F4809165008195809375
:100F000065002EDBC3C0113009F093C0A99711F41E
:100F100010936500662391F080919E0070E061500F
:100F2000710990E0EDD76091B90070E01AD86111B5
:100F300001C061E06093E0006093C1008091E00037
:100F40009091E100282F30E0291B310960919C002D
:100F500070919D006F5F7F4F70939D0060939C0028
:100F60002115310509F492C037FF05C0933830F0E0
:100F700040E450E005C040E052E002C040E051E0F3
:100F80005695479537FF02C02F5F3F4F3595279500
:100F900021153105A9F74617570708F077C08917BB
:100FA00010F48FEF03C0981710F481E0890F7FEFE2
:100FB000780F272F30E0A9014F535F4FFA0164915A
:100FC000791738F499B5911104C06F3F11F469BDD8
:100FD0000CC099B5961718F499B59F5F05C099B5DF
:100FE000691718F499B5915099BD255D3F4FF901E6
:100FF000949168B5691718F498B59F5F05C068B5F6
:10100000961718F498B5915098BD99B5FA01449186
:1010100094130AC098B5F9012491921305C0C091A8
:10102000E000D2DAC093E00010929D0010929C0084
:101030002DC01530A1F48091E100823438F190E0A8
:101040008C1B9D0B282F813491052CF0873991053D
:1010500018F026E901C021E42093E00017C0163003
:10106000B9F49091E1008091C100981778F4C90F0C
:10107000D11D90E08C179D0734F0C134D10524F4C4
:10108000C1E4D0E001C0EC01C093E00000E056C034
:10109000173071F49091E0008091E100891710F40D
:1010A0008F5F03C0981790F781508093E000EECFD8
:1010B000133C79F481E0D11080E08093BD00CFD95A
:1010C0004FDACCDA8091E10090E034D980937B0054
:1010D000C4CE011132C0133B41F4CD2BB9F6EE2042
:1010E00011F086E9F82E8F2D04C0133E21F4809173
:1010F0007B00A3DA23C0153C41F480E065DA60E0B0
:1011000070E089E69CE0D5DB19C0173B29F460E06C
:1011100070E081E196E00FC01A3C39F48091E10063
:101120008093C0009CD98CDA09C01A3B31F460E08E
:1011300070E08BE196E0A5DB01C001E0802FDF913C
:10114000CF911F910F91FF90EF90DF90CF90BF90C4
:10115000AF909F9008958CE287B910920A01109287
:101160000B0186B1886486B9089510920C0124B1F0
:1011700095B13091DF002295269526952370892F11
:1011800090E0880F991F880F991F820F911D830F80
:101190008093DF0080910101882309F40BC1109234
:1011A000010180910A019091E200992319F037988A
:1011B00010920A01811143C080917E00882349F07A
:1011C0006091060170910701709303016093020121
:1011D00004C06091020170910301605F7F4FA6E03F
:1011E00076956795AA95E1F780E098E5A6D6809177
:1011F0007D0090E00297680F791F76956795609360
:1012000000018091B200882311F0815007C06D3138
:1012100038F460E070E084E0BBD785E08093B200F2
:101220008091E2008111BDC08FEA87B981E080938F
:101230000A0110920B0186B1886486B9B2C0813070
:1012400009F0AFC080917E00811143C080910401FC
:101250009091050140969C0145E0369527954A9569
:10126000E1F7A091FD00A901569547950A2E000CC3
:10127000BB0BCD0183519140840F951F9093FF00CC
:101280008093FE008091A100E82FF0E0EE0FFF1F99
:10129000EE55FF4F40815181B901641B750B3183BD
:1012A00020838F5F87708093A100CB01880F991FE7
:1012B000880F991F40917C0050E04D5E5E4F4A1BA5
:1012C0005B0B440F551F841B950B820F931F23E06C
:1012D0001CC08091080190910901909305018093B1
:1012E0000401409635E0969587953A95E1F7E2EA54
:1012F000F0E08193919320E0E23BF207D1F7A6CF93
:10130000009709F00196215029F018161906C4F724
:101310000197F9CF18161906E4F477FD39C020912A
:10132000A00012160CF1880F991FBC0163507109BF
:1013300077FF02C06F5F7F4F75956795161617068A
:1013400014F061E070E088E1861B8093A00085E0E6
:1013500026C08C3F2FEF9207DCF477FF19C0209155
:10136000A00027FF05C02450281B2093A00018C010
:1013700024EE281B2093A000209100012F3180F043
:101380006CEF7FEF681B790B7595679586E007C05A
:10139000809100018E3120F060E070E087E0F8D6A7
:1013A000DADE80917E00882329F080917E008150D2
:1013B00080937E0008950F931F93CF931092E500C2
:1013C00080913D0190913E019C012F5F3F4F882706
:1013D0009078822B932B90933E0180933D01C09196
:1013E000E3004AD7C81729F11092E2008093E30086
:1013F00090913F01882359F0892F80699F709F3019
:1014000009F08F5F80933F0180E090E00DC0892F4D
:101410008F7E95FD02C0806801C0806C80933F0183
:1014200080913D0190913E0103D710923E011092B0
:101430003D0100913D0110913E018091E200882321
:1014400079F0B80183E0A4D6BCD60F731127012B25
:1014500009F044C010929F007EDE87EE86B92EC050
:10146000C0913F018C2F807F803B19F460E070E0D9
:1014700001C0B80181E08CD6C4FF12C0C5FF02C014
:10148000C8010CC008311105C8F010923E0110923D
:101490003D01C062C0933F0180E090E0C9D60EC01C
:1014A000CC2361F0C5FD09C00231110538F0C064DC
:1014B000C0933F0180E090E0BBD6BED680919F00F4
:1014C000811106C086B1886486B981E080930101EC
:1014D00080919F008F5F8F7180939F00CF911F91AC
:1014E0000F91089580910C0181113FDE8091E500FC
:1014F000811161CF0895CF92DF92EF92FF920F9307
:101500001F93CF93DF93EC0110E800E088E0E82E12
:1015100087E0F82E92ECC92EDD24D394209709F1B0
:101520008091C40081111FC08091E100853040F49A
:1015300082E00FB6F89416BD86BD0FBEC60106C088
:101540000FB6F89416BD06BD0FBEC7010197F1F79F
:101550000FB6F89416BD06BD0FBEC4DF32D6219774
:10156000DDCF81E001C080E0DF91CF911F910F912D
:10157000FF90EF90DF90CF900895CF93C82F8823EE
:1015800081F089E121D886EA90E0B5DF80E01CD8BF
:101590008AEF90E0B0DFC150A1F78AE992E0CF91E5
:1015A000AACF89E111D888E090E0A5DF80E00CD8CF
:1015B0008AEF90E0A0DFF1CFCF93DF9364E6B1D460
:1015C000282F892F6AE0ADD4EC01222341F0822F2D
:1015D000D4DF8C2FD2DF8D2FDF91CF91CECFC111F1
:1015E000F8CFF9CFDF92EF92FF920F931F93CF9333
:1015F000DF93D82F8B01C0916B0081E08093B50001
:10160000C33009F0D3C0F090BA008D2F56D8FF2018
:1016100051F08091BA00811106C060E070E08EEE5A
:1016200094E047D9C3C0D83021F481E080936300AF
:10163000BFC0D23C19F41092BA00C8C0D13BC1F46B
:1016400090916200012B49F49E3610F08FEF03C099
:10165000923018F481E08093630080916300890FD9
:1016600011F481E02BC18F3608F428C18EE626C123
:10167000D13E31F480916300819580936300DCC09A
:10168000D23B61F481E080936300809162008230FC
:1016900008F4DAC0815080936200D6C0D13009F0DE
:1016A000E4C00932110511F4D0936300D090990081
:1016B0008D2D880FD7FC809590E067E070E020D4F6
:1016C000292FE09098008E2D880FE7FC8095D0910F
:1016D00061006D2F70E090E013D4290FF090970017
:1016E0008F2D880FF7FC8095C09160006C2F70E003
:1016F00090E006D4920F6091620070E0690F711D56
:101700008091BA00813091F48091B7009091B80037
:1017100025E0969587952A95E1F724E730E0A90121
:10172000481B590BCA01ECD3B90107D4862F4CD7FB
:1017300000FD05C0AAD58170D80ED0929900809185
:101740009600E80EE0929800A0D565E2EAD3F90E83
:10175000F09297009AD58F7329F497D56DE0E1D375
:1017600090939600DD2331F090D58F7319F4D1500A
:10177000D09361008AD5811107C087D56BE0D1D3A2
:101780009093610010929800C33030F07ED58F7135
:1017900019F4C150C093600078D58F7709F079C0F3
:1017A00074D566E0BED39093600073C0D83021F446
:1017B00081E08093640084C0D13C31F460E070E04B
:1017C0008EEE94E076D87CC0D23C49F48C2F90E029
:1017D000019665E070E0C5D380936B004BC0D13BB0
:1017E00049F5C23090F400FD6BC0EC2FF0E0E759F2
:1017F000FF4F808190916400891B883020F08F3FDB
:1018000091F58EEF30C088E02EC0C43009F058C08A
:101810009091680080916400890F823010F482E01A
:1018200003C0893708F088E78093680080916800DA
:10183000CBD646C0D13E31F480916400819580932F
:10184000640018C0D23BA1F481E080936400C230F0
:1018500060F500FD35C0EC2FF0E0E759FF4F8081C7
:101860008F3F71F18F5F80832BC0D13C09F4A6CFED
:10187000D23E11F4F4D524C0D53C39F460E070E0D8
:1018800089E69CE016D880E0D3CFD13011F081E01A
:1018900018C00932110519F481E080936400809129
:1018A000DF00080F0093DF000BC0C43049F48091C3
:1018B0006800833008F4BACF8150B6CF80936200BD
:1018C00080E0DF91CF911F910F91FF90EF90DF901B
:1018D00008950F931F93CF93DF93D82F8B018830F8
:1018E00031F48091B500813011F488E07BDE8D2FDA
:1018F0008079803959F481E08093B400C091B500BB
:10190000C1110AC080917B005FD621C0803831F4BC
:101910001092B40080E058D6C0E019C0D130B1F4C4
:10192000C091B400CC2351F08091B5008130A1F773
:10193000B801DF91CF911F910F9154CE0733114021
:1019400058F3D093E20080E033D601C0C1E08C2F81
:10195000DF91CF911F910F9108951F920F920FB6B3
:101960000F9211242F933F938F939F93AF93BF9325
:10197000EF93FF9380910B018823E9F0E0910A0136
:1019800024B135B1F0E0EE0FFF1FDF01AA5FBE4FBB
:101990002D933C93EE5FFE4F8081918182179307D8
:1019A00008F401962817390708F40197918380837A
:1019B00081E080930C0181E080930B01FF91EF9116
:1019C000BF91AF919F918F913F912F910F900FBE3B
:1019D0000F901F9018951F920F920FB60F9211241F
:1019E0008F9381E08093E5008F910F900FBE0F9051
:1019F0001F9018951F920F920FB60F9211248F937C
:101A000081E08093E4008F910F900FBE0F901F90A4
:101A10001895F89484B7877F84BF0FB6F894A8957B
:101A200081B5886181BD11BC0FBEB89A81E083BFCA
:101A300081EA8ABDB99A88E088BB85BB8BB7806292
:101A40008BBFA89581B5886181BD80E481BD83DBB2
:101A500087EE86B9789481E0F9D360E070E087E69C
:101A600094E00FD71092C40004B603FC08C0F894A9
:101A700080E091E089D2853A51F178949BC0C0E032
:101A80008C2FA2D583E190E036DD8C2F86959CD5F6
:101A900083E190E030DDF0D3882381F0CF5FC03464
:101AA00079F765E181E0BDD4DAD4C6E98C2F8CD515
:101AB00084E090E020DDC150C9F7D9CFCC23B9F242
:101AC0008C2F82D58DE090E016DDC150F7CF06EC6B
:101AD00010E0C1E0D1E0CE0157D2F80181938F012F
:101AE0002196CA31F1E0DF07B1F778948091C60002
:101AF0008093BD008091C700809374008091C800DE
:101B0000809371008091C900809375008091CA0014
:101B1000809372008091CB0080936F008091CC0005
:101B2000809376008091CD00809373008091CE00E9
:101B3000809370008091CF0080937A008091D000D4
:101B40008093BE008091D1008093BC008091D20030
:101B5000809379008091D3008093C0008091D4005D
:101B60008093BF008091D50080936B008091D60058
:101B7000809369008091D70080936A008091D8009B
:101B8000809368008091D90080936C008091DA0086
:101B900080937C008091DB008093FD008091DC00CD
:101BA00080937D008091DD0080936D008091DE0048
:101BB0008093B600F894C0E0D0E0CE01E5D1853A3C
:101BC00059F4D093C300C093C200CE010196DCD17A
:101BD0008093C50081E005C02296CE3FD10569F70C
:101BE00080E07894882321F08091C50080937B0069
:101BF00043D38823E9F061E070E08EEB96E041D6B4
:101C000043E4242E52E0352E67EE462E552453949D
:101C1000CC24C394D12CECEF6E2EE3E07E2EFEEEAE
:101C2000AF2EF4E0BF2EAAE28A2EA0E09A2E13C0B7
:101C300060917B0070E0E1CFFAE0823F9F0709F0FE
:101C40007EC0C0916B00C23009F4A4C008F487C004
:101C5000C43009F4F9C0B5D28091E8009091E90050
:101C6000009749F06091E6007091E70022D610924B
:101C7000E9001092E8008091E200882309F445C051
:101C800080E0A2D4A89581B5886181BD21BC379838
:101C9000F3D28111FDCFD0D28BB780628BBF10926F
:101CA0000C011092E5001092E4008091E20088237C
:101CB000F9F085B7877E806185BF85B7806285BF73
:101CC000889585B78F7D85BF8091E4008111109242
:101CD000E20080910C01882329F050927E005092FE
:101CE000010143DA8091E5008823F9F264DBDDCF5E
:101CF00030927E008BB78F7D8BBF2DDA46B8A895CA
:101D000081B5886181BD80E481BDECDB1092C400A7
:101D10008091FB009091FC0022E08B30920709F04B
:101D20008BCFCEE1D0E0FE018491805326DC8CE2A3
:101D300091E0E1DB21968C169D06A9F7AAC02CE064
:101D40008936920709F09AC08091B500813009F078
:101D5000CCC08091B400882309F4C7C072CFEC2FA7
:101D6000F0E0E759FF4FD08186E92ED4C11109C0B8
:101D7000DA3220F4C3010197F1F707C081E090E067
:101D800003C08D2F869590E0B6DB80E01DD48D2FAB
:101D900090E0A9C07AD28F73E82EF12C76D267E05A
:101DA000C0D0E60102C0CC0FDD1F9A95E2F76DD2DC
:101DB00065E0B7D0F60102C0EE0FFF1F9A95E2F77B
:101DC000CE0FDF1F62D290E0BE01CBD0C80FD91F6B
:101DD000C739D10514F0C6E9D0E08C2FF5D3C7017F
:101DE0008ADB8E0133E0159507953A95E1F70111ED
:101DF00001C001E010E0C7017EDBC01BD10BD7FFA3
:101E000002C0C0E0D0E08C2FDFD33FD2837031F42A
:101E1000C70171DBCE0195958795D6D3C230D10528
:101E200054F733D26DE07DD0E60102C0CC0FDD1F48
:101E30009A95E2F72AD290E0BE017FD0C80FD91F51
:101E400080E0C2D3CE014FC0C0916800CC0FC7392B
:101E500008F0C6E9D4E08C2FB7D385E090E04BDBE7
:101E600080916800B1D381E490E045DBD15099F7CF
:101E700080ED92E040DB80E0A7D3EDCEF4E0843B40
:101E80009F0781F48091000197DB80917A0088237D
:101E900081F0B092E900A092E8001092E700109261
:101EA000E600D9CE24E0843D920731F48091FE0013
:101EB00083DB88EE93E017C08D589440B1F4809195
:101EC000E3008111C8CE80917B007ED384E690E050
:101ED00012DB80E079D380916C0090E068EE73E0D3
:101EE0000FD08456910907DBB6CE85B7877E85BFB4
:101EF00085B7806285BF889585B78F7D85BFABCE5E
:101F00000024552704C0080E591F880F991F0097F9
:101F100029F076956795B8F37105B9F7802D952F5F
:101F20000895991B79E004C0991F961708F0961B35
:101F3000881F7A95C9F780950895AA1BBB1B51E1AC
:101F400007C0AA1FBB1FA617B70710F0A61BB70B29
:101F5000881F991F5A95A9F780959095BC01CD01CE
:101F6000089597FB072E16F4009406D077FD08D04D
:101F7000E4DF07FC05D03EF4909581959F4F0895CE
:101F8000709561957F4F0895E199FECF9FBB8EBB01
:101F9000E09A99278DB30895262FE199FECF9FBB34
:101FA0008EBBE09A01970DB2021639F01CBA2DBB18
:101FB0000FB6F894E29AE19A0FBE0895F894FFCF15
:101FC000060B18010101000441294303020D01071A
:101FD00005787896010A0A78010101412D070274FB
:101FE0000071006E0000010201000000000000010D
:061FF000000000000000EB
:00000001FF
